:020000040000FA
:100000000000022818309A0001309B008030000068
:1000100000009E2000000000831200009D001B08CD
:100020009C001A309E0001309F00831200001C08C3
:10003000A0001D08A100FF309C07031C9D032108A0
:10004000200403199A2804301E07A000A101A10D65
:100050001F08A10720089A0021089B00803000009B
:1000600000009E200000000083120000A3001B0877
:10007000A2001E089A001F089B00803000000000AC
:100080009E200000000083120000A500A1001B08B4
:10009000A000A40002301E07A000A101A10D1F08AE
:1000A000A10720089A0021089B0080300000000072
:1000B0009E200000000083120000A100A7001B0882
:1000C000A600A000831200002208A6002308A700B3
:1000D000FF30A207031CA303270826040319932853
:1000E00024089A0025089B00803000000000BF20F3
:1000F0000000000083120000A600200883120313F2
:1001000084008313831200002118831726088312AA
:100110000313800083120000A40A0319A50AA00A91
:100120000319A10A62280630831200009E070318F3
:100130009F0A152800000000D2280800003A031981
:10014000A628803A0319B0289B0100341A088400BD
:1001500083131B18831700089B00840A00080800FB
:1001600000000000CD2099009A0F9B039B0A00001D
:100170000000CD20980019089B0018080800003ADC
:100180000319C628803A0319CD2800341A088400C0
:1001900083131B188317000808001B088A001A081D
:1001A000820008000030AF00FD30AE008030B000AB
:1001B0002E089A002F089B003008AC001B08AB00EB
:1001C0001A08AA002A089A002B089B002C08BF20B6
:1001D000AD002D080319F4282D080F21AA0A0319D0
:1001E000AB0A0319AC0AE22883127208AE00AE18FB
:1001F000F42871080F21F4280800483465346C3461
:100200006C346F342034663472346F346D3420347F
:1002100050344934433421340D340A340034A800B6
:1002200083127208A900291810292808F000080074
:1002300001340034203401343134003401340034CA
:02024000003488
:00000001FF
